:020000000628D0
:080008000B110900831685109D
:10001000061283120130003C03192B280530990089
:1000200001309A0080309B008A200230A100B92064
:1000300005309700013098007B2005309C0001308E
:100040009D00A02006160130A100B9200612013043
:10005000A100B9200A280D088F006E308E00000024
:10006000000000000000000000008E0B2F288F0B06
:100070002D28080011088C00D53E00300318013EE1
:100080008A000C08D420940011088C00DE3E003059
:100090000318013E8A000C08DD209500100884003A
:1000A000000814048000FF3093001308003C013066
:1000B000031900019303003C03195F2855280930F8
:1000C00096000310031C692800081404800003181C
:1000D0006C2800081505800086309300930B6E286D
:1000E0000000920C960B6228000814048000013076
:1000F0008D002B200800170890001808910055303B
:1001000092003A20170890001808910000309200E1
:100110003A200800190890001A0891005530920002
:100120003A20190890001A089100033092003A20F2
:10013000190890001A0891001B0892003A20080044
:100140001C0890001D089100553092003A201C08B0
:1001500090001D089100013092003A2008001E080E
:100160009F001430A00000000000A00BB3289F0BDC
:10017000B1282108003C013003190001003C03199B
:10018000D3280030A2000A302202013003180001F7
:10019000003C0319D02864308D002B20A20AC3280C
:1001A0002108A103B928080082070134023404346D
:1001B000083410342034403480348207FE34FD3457
:0C01C000FB34F734EF34DF34BF347F34FD
:00000001FF
